:10000000592864001120031801281C200830A3007F
:100010001D201120A20C0C28A30B08281D2022084B
:10002000080038088400360884178004841300050B
:1000300035193606FF3E08003517350D0639A00084
:100040002B20A100A00A2B20351F38283513A00033
:1000500002304F20382800308A00200882070134FF
:1000600075340334153400343C340C34D934A101D4
:10007000E83EA000A109FC30031C4128A00703189A
:100080003E28A0076400A10F3E2820184728A01C86
:100090004B2800004B2808000310A10CA00CFF3EC9
:1000A00003184C2820085428831303138312640078
:1000B0000800FF2383168F008312831607309F00EA
:1000C0002F30850083120512831605128312BA01A0
:1000D000BB01BC01BB01BA010508BB000730BB0571
:1000E0003B08073C031C83287720BA008328003094
:1000F0008A003B0882074134423443344434453457
:100100004634473448340530B8002030B600073054
:10011000B50001203A02031D89280120BC006400BB
:100120003C08303C03199A2864003C08313C031910
:100130009F286A2805128316051283126A2805165D
:080140008316051283126A28E0
:02400E006C3F05
:00000001FF
